:0200000480007A
:100000006F00C004732F2034930F8000630AFF0336
:10001000930F90006306FF03930FB0006302FF038A
:10002000170F0080130F0FFE63040F0067000F000F
:10003000732F203463540F006F004000136E9E53E3
:10004000171F00002320CFFD6FF09FFF732540F1A5
:100050006310050073251030635805000F00F00F82
:10006000130E100073000000130E00009702000032
:10007000938282F973905230735020307350303035
:1000800073504030970200809382C2F7638C020065
:10009000739052109302B01A739022307323203061
:1000A000E39E62F873500030970200009382420191
:1000B00073901234732540F173002030130E20002A
:1000C000930000001301100063C620006318C02BCA
:1000D0006316C001E3CE20FE6312C02B130E300066
:1000E0009300F0FF1301100063C620006318C029BD
:1000F0006316C001E3CE20FE6312C029130E400038
:100100009300E0FF1301F0FF63C620006318C027CF
:100110006316C001E3CE20FE6312C027130E500009
:10012000930010001301000063C420006314C00199
:100130006316C025E3CE20FE130E6000930010006E
:100140001301F0FF63C420006314C0016318C023CF
:10015000E3CE20FE130E70009300F0FF1301E0FFCA
:1001600063C420006314C001631AC021E3CE20FEE3
:10017000130E8000930010001301E0FF63C4200001
:100180006314C001631CC01FE3CE20FE130E900059
:1001900013020000930000001301F0FF63C0201E53
:1001A0001302120093022000E31652FE130EA00069
:1001B00013020000930000001301F0FF1300000081
:1001C00063CE201A1302120093022000E31452FEA1
:1001D000130EB00013020000930000001301F0FFA3
:1001E000130000001300000063CA2018130212005D
:1001F00093022000E31252FE130EC000130200000F
:1002000093000000130000001301F0FF63C82016E4
:100210001302120093022000E31452FE130ED000CA
:100220001302000093000000130000001301F0FF10
:100230001300000063C42014130212009302200074
:10024000E31252FE130EE0001302000093000000C0
:1002500013000000130000001301F0FF63C0201220
:100260001302120093022000E31252FE130EF0005C
:1002700013020000930000001301F0FF63C0201080
:100280001302120093022000E31652FE130E000127
:1002900013020000930000001301F0FF13000000A0
:1002A00063CE200C1302120093022000E31452FECE
:1002B000130E100113020000930000001301F0FF61
:1002C000130000001300000063CA200A130212008A
:1002D00093022000E31252FE130E200113020000CD
:1002E00093000000130000001301F0FF63C8200812
:1002F0001302120093022000E31452FE130E300189
:100300001302000093000000130000001301F0FF2F
:100310001300000063C420061302120093022000A1
:10032000E31252FE130E400113020000930000007E
:1003300013000000130000001301F0FF63C020044D
:100340001302120093022000E31252FE93001000E9
:10035000634A100093801000938010009380100077
:10036000938010009380100093801000930E300053
:10037000130E50016394D001631CC0010F00F00FF5
:1003800063000E00131E1E00136E1E00730000009B
:100390000F00F00F130E100073000000731000C068
:1003A000000000000000000000000000000000004D
:1003B000000000000000000000000000000000003D
:0403C0000000000039
:1010000000000000000000000000000000000000E0
:1010100000000000000000000000000000000000D0
:1010200000000000000000000000000000000000C0
:1010300000000000000000000000000000000000B0
:081040000000000000000000A8
:040000058000200057
:00000001FF
